:020000040000FA
:04000000EE303A287C
:08000800A000030EA100831209
:1000100005191028831601178312B23081002B288E
:1000200083160113831203140B190310A80DA90DD5
:10003000AA0DAB0DAC0DAC16FF302C02031D2B2806
:10004000FA302B02031D2B2831152A08AF0029088E
:10005000AE002808AD008B100B11210E8300A00EFE
:04006000200E090065
:0C007400203084008001840A80300402E7
:10008000031C3C281230B000092283160C30850571
:1000900087018312850187010730990000309A009B
:1000A000103083168E008312603083168F00831207
:1000B0000030831691009F008312C83083168100A0
:1000C000831231309000003083168C008312103080
:1000D0008B00892381018E018F010B118B100B1076
:1000E0008C018B17812031198420B30B7F280310DA
:1000F00085190314B90DF030390203195721F02383
:10010000722864003210080031110130B7008B13DF
:1001100020303707371A313E83169B001C141A080B
:100120008312A40010303707371A313E83169B0024
:100130001C141A088312A300A6000230A606003081
:100140003707371A313E83169B001C141A08831296
:10015000A200A7000130A7068B17321CB528220980
:100160000339A200A309A409A50924082F02031D2D
:10017000512923082E02031D512922082D02031D97
:10018000512901303702031DCA283D18CA283D14E1
:100190003E14242202303702031DD328BD18D32871
:1001A000BD143E14362203303702031DDC283D19EE
:1001B000DC283D153E14482204303702031DE52893
:1001C000BD19E528BD153E145A2205303702031D1E
:1001D000EE283D1AEE283D163E146C2206303702FA
:1001E000031DF728BD1AF728BD163E147D220730DF
:1001F0003702031D00293D1B00293D173E148E22A6
:1002000008303702031D0929BD1B0929BD173E14FB
:100210009F2209303702031D12295E1812295E142D
:100220003E14B0220A303702031D1B29DE181B2999
:10023000DE143E14C1220B303702031D24295E193F
:1002400024295E153E14D2220C303702031D2D29BD
:10025000DE192D29DE153E14E3220D303702031D71
:1002600036295E1A36295E163E14F4220E30370205
:10027000031D3F29DE1A3F29DE163E1405230F30E9
:100280003702031D48295E1B48295E173E141623BA
:1002900010303702031D5129DE1B5129DE173E1491
:1002A0002723B70A0F3037020318080087280130C8
:1002B000B600B300B400B500B70085018701B113E3
:1002C0008120B30BAF29031085190314B90DF03049
:1002D00039020319DC29B40BAF29013037020319A5
:1002E00039230230370203193E2303303702031942
:1002F000432304303702031948230530370203191A
:100300004D230630370203195223073037020319F1
:1003100057230830370203195C23093037020319C9
:1003200061230A303702031966230B3037020319A1
:100330006B230C303702031970230D303702031979
:1003400075230E30370203197A230F303702031951
:100350007F2310303702031984239630B400311DF7
:1003600060293111321CB9292D090339AD00AE09BC
:10037000AF092F1C60298E018F010C1C60290C1005
:100380002E1E60298B1320303707371A313EBB00F1
:100390002F08BA00F42110303707371A313EBB005E
:1003A0002E08BA00F42100303707371A313EBB005F
:1003B0002D08BA00F4218B1785018701B70AB60111
:1003C0000F303702031C6029892308003E1C0800F7
:1003D0003E101030BB003D08BA00F4213030BB00A5
:1003E0005E08BA00F42108008B133A0883161C1526
:1003F0009A0083123B0883169B0055309D00AA305B
:100400009D009C1464009C18022A1C1183128B17F7
:100410000800831610309B001C141A088312BD00BC
:10042000831630309B001C141A088312DE00FF3044
:10043000C800CA15CB15CC15CD15CE15CF15D015C6
:10044000D115D215D31508000130BD050030DE05E9
:100450000530C405C0000030C200C6004030C505EC
:10046000C1004030C300C7005F1008000230BD0566
:100470000030DE053530C405C0000030C200C600C3
:100480004030C505C1004030C300C7005F10080000
:100490000430BD050030DE050530C405C000043061
:1004A000C200C6004030C505C1004030C300C700CF
:1004B0005F1008000830BD050030DE054830C40577
:1004C000C0000030C200C6008030C505C1008030C9
:1004D000C300C7005F1008001030BD050030DE0506
:1004E000CA30C405C0008030C200C6008030C505D7
:1004F000C1008030C300C70008002030BD050030B7
:10050000DE052930C405C0000030C200C6004030FE
:10051000C505C1004030C300C70008004030BD051C
:100520000030DE051930C405C0000030C200C6002E
:100530004030C505C1004030C300C700080080300E
:10054000BD050030DE05AA30C405C0008030C20001
:10055000C6008030C505C1008030C300C700080058
:100560000030BD050130DE059A30C405C000803082
:10057000C200C6008030C505C1008030C300C7007E
:1005800008000030BD050230DE053930C405C0006A
:100590000030C200C6004030C505C1004030C30075
:1005A000C70008000030BD050430DE05B230C405C8
:1005B000C0008030C200C6008030C505C100803058
:1005C000C300C70008000030BD050830DE0522303A
:1005D000C405C0000230C200C6004030C505C100DD
:1005E0004030C300C70008000030BD051030DE05F4
:1005F0003230C405C0001230C200C6004030C5050C
:10060000C1004030C300C70008000030BD052030E5
:10061000DE050830C405C0000030C200C600C0308E
:10062000C505C100C030C300C70008000030BD05CB
:100630004030DE050030C405C0000030C200C600F6
:100640000030C505C1000030C300C70008000030FD
:10065000BD058030DE050030C405C0000030C2009A
:10066000C6000030C505C1000030C300C700080047
:100670000800113085061030870608001130850605
:1006800016308706080011308506103087060800EE
:100690000230850609308706080022308506293099
:1006A00087060800123085061430870608001230CD
:1006B0008506123087060800223085062C30870612
:1006C0000800223085062A30870608001230850689
:1006D000163087060800203085062E308706080071
:1006E0002030850614308706080020308506163035
:1006F000870608000230850618308706080000309B
:100700008506003087060800003085060030870621
:1007100008003D182422BD1836223D194822BD1973
:100720005A223D1A6C22BD1A7D223D1B8E22BD1B12
:100730009F225E18B022DE18C1225E19D222DE1975
:10074000E3225E1AF422DE1A05235E1B1623DE1B4B
:1007500027230800B601B301B4013C1CB22BBC0135
:10076000BC14B42BBC013C143C08B6006400B82B8C
:10077000B92BBA2BBB2BBC2BFF30B41B8500B41F8D
:100780008501B30BB62BB40BB62B0310B60CB60811
:10079000031DB62B0030BB003C08BA00F421080052
:1007A00005125C180516DC1C8512DC1885165C1D0C
:1007B00005105C190514DC1D8510DC1985145C1E00
:1007C00087105C1A8714DC1E0711DC1A07155C1FE2
:1007D00007105C1B0714DC1F8712DC1B8716080040
:1007E0008F08031908008F0178308E00C80F2E2E55
:1007F000C80ADF19222C441C222C461C132CCA1CAC
:10080000042CCA014A15302C4A1D092CCA01CA15EC
:10081000302CCA1D0E2CCA014A16302C4A1E302C10
:10082000CA01CA14302C4A1D182CCA014A16302C91
:10083000CA1D1D2CCA014A16302C4A1E302CCA0172
:10084000CA14302CCA1C272CCA014A15302C4A1D48
:100850002C2CCA01CA15302C4A1E302CCA014A154C
:10086000DF19592CC41C592CC61C4A2CCB1C3B2C00
:10087000CB014B15672C4B1D402CCB01CB15672CA6
:10088000CB1D452CCB014B16672C4B1E672CCB0187
:10089000CB14672C4B1D4F2CCB014B16672CCB1D5B
:1008A000542CCB014B16672C4B1E672CCB01CB1461
:1008B000672CCB1C5E2CCB014B15672C4B1D632C7E
:1008C000CB01CB15672C4B1E672CCB014B15DF19C9
:1008D000902C441D902C461D812CCC1C722CCC01DC
:1008E0004C159E2C4C1D772CCC01CC159E2CCC1D70
:1008F0007C2CCC014C169E2C4C1E9E2CCC01CC1476
:100900009E2C4C1D862CCC014C169E2CCC1D8B2C69
:10091000CC014C169E2C4C1E9E2CCC01CC149E2C33
:10092000CC1C952CCC014C159E2C4C1D9A2CCC012A
:10093000CC159E2C4C1E9E2CCC014C15DF19C82CBE
:10094000C41DC82CC61DB92CCD1CAA2CCD014D151B
:100950005F13D62C4D1DAF2CCD01CD15D62CCD1D42
:10096000B42CCD014D16D62C4D1ED62CCD01CD1458
:10097000D62C4D1DBE2CCD014D16D62CCD1DC32C15
:10098000CD014D16D62C4D1ED62CCD01CD14D62C16
:10099000CD1CCD2CCD014D15D62C4D1DD22CCD010D
:1009A000CD15D62C4D1ED62CCD014D15DF19012DA0
:1009B0005F1B012D441E012D461EF22CCE1CE32C84
:1009C000CE014E150F2D4E1DE82CCE01CE150F2D4C
:1009D000CE1DED2CCE014E160F2D4E1E0F2DCE012D
:1009E000CE140F2D4E1DF72CCE014E160F2DCE1D01
:1009F000FC2CCE014E160F2D4E1E0F2DCE01CE1407
:100A00000F2DCE1C062DCE014E150F2D4E1D0B2D7C
:100A1000CE01CE150F2D4E1E0F2DCE014E15DF1916
:100A2000382DC41E382DC61E292DCF1C1A2DCF01DE
:100A30004F15462D4F1D1F2DCF01CF15462DCF1D14
:100A4000242DCF014F16462D4F1E462DCF01CF141A
:100A5000462D4F1D2E2DCF014F16462DCF1D332D68
:100A6000CF014F16462D4F1E462DCF01CF14462DD8
:100A7000CF1C3D2DCF014F15462D4F1D422DCF01CF
:100A8000CF15462D4F1E462DCF014F15DF196F2D67
:100A9000441F6F2D461F602DD01C512DD0015015C5
:100AA0007D2D501D562DD001D0157D2DD01D5B2DD7
:100AB000D00150167D2D501E7D2DD001D0147D2DDE
:100AC000501D652DD00150167D2DD01D6A2DD001F1
:100AD00050167D2D501E7D2DD001D0147D2DD01CA3
:100AE000742DD00150157D2D501D792DD001D015BC
:100AF0007D2D501E7D2DD0015015DF19A62DC41F50
:100B0000A62DC61F972DD11C882DD1015115B42DAE
:100B1000511D8D2DD101D115B42DD11D922DD10195
:100B20005116B42D511EB42DD101D114B42D511D27
:100B30009C2DD1015116B42DD11DA12DD1015116DD
:100B4000B42D511EB42DD101D114B42DD11CAB2D17
:100B5000D1015115B42D511DB02DD101D115B42D98
:100B6000511EB42DD1015115DF19DE2D451FDE2D8B
:100B7000471FCF2DD21CC02DD2015215DF13EC2DF3
:100B8000521DC52DD201D215EC2DD21DCA2DD20178
:100B90005216EC2D521EEC2DD201D214EC2D521D0A
:100BA000D42DD2015216EC2DD21DD92DD2015216C0
:100BB000EC2D521EEC2DD201D214EC2DD21CE32DC3
:100BC000D2015215EC2D521DE82DD201D215EC2D7B
:100BD000521EEC2DD2015215DF19172EDF1B172ED6
:100BE000C51F172EC71F082ED31CF92DD30153156F
:100BF000252E531DFE2DD301D315252ED31D032ED7
:100C0000D3015316252E531E252ED301D314252E82
:100C1000531D0D2ED3015316252ED31D122ED30195
:100C20005316252E531E252ED301D314252ED31C47
:100C30001C2ED3015315252E531D212ED301D31560
:100C4000252E531E252ED3015315E6214008C4003E
:100C50004108C5005F18DF145F1CDF104808C90099
:100C60000C304A05031D05120C304B05031D85127F
:100C70000C304C05031D05100C304D05031D85106F
:100C80000C304E05031D87100C304F05031D071156
:100C90000C305005031D07100C305105031D871241
:100CA0000C305205031D07120C305305031D87112C
:100CB00049080E020318882E12304A05031D051636
:100CC00012304B05031D851612304C05031D05140B
:100CD00012304D05031D851412304E05031D871477
:100CE00012304F05031D071512305005031D071460
:100CF00012305105031D871612305205031D0716C9
:100D000012305305031D8715FF30480203190800F0
:100D10008F08031D0800812049080E02031C882E3D
:100D200018304A05031D051206304A05031D051635
:100D300018304B05031D851206304B05031D851623
:100D400018304C05031D051006304C05031D051415
:100D500018304D05031D851006304D05031D851403
:100D600018304E05031D871006304E05031D8714ED
:100D700018304F05031D071106304F05031D0715D9
:100D800018305005031D071006305005031D0714C9
:100D900018305105031D871206305105031D8716B3
:100DA00018305205031D071206305205031D0716A1
:100DB00018305305031D871106305305031D871591
:020DC000080029
:084000000E000300050007009B
:02400E00CC33B1
:10420000010078007A007C007E007B0079007F004E
:104210007D007A0078007E007C007D007F007900C0
:104220000200F200F600FA00FE00F200F600FA00CA
:10423000FE00F200F600FA00FE00F200F600FA00BE
:10424000FF00050005000500050009000900090040
:1042500009000D000D000D000D00110011001100EE
:104260000100FF00FF00FF00FF00FF00FF00FF0054
:10427000FF00FF00FF00FF00FF00FF00FF00FF0046
:10428000FF007B00FF00FF00FF00FF00FF00FF00BA
:10429000FF00FF00FF00FF00FF00FF00FF00FF0026
:1042A000FF00FE00FF00FF00FF00FF00FF00FF0017
:1042B000FF00FF00FF00FF00FF00FF00FF00FF0006
:1042C000FF001100FF00FF00FF00FF00FF00FF00E4
:1042D000FF00FF00FF00FF00FF00FF00FF00FF00E6
:1042E000FF00FF00FF00FF00FF00FF00FF00FF00D6
:1042F000FF00FF00FF00FF00FF00FF00FF00DD00E8
:00000001FF
